:1000000012C0B2C0BCC01FC01EC01DC01CC01BC0DF
:100010001AC019C018C017C016C015C014C013C02C
:1000200012C011C010C011241FBECFE5D4E0DEBF46
:10003000CDBF10E0A0E6B0E001C01D92A736B10729
:10004000E1F7A8D0E3C0DCCFBB9A88B388BB89E0D6
:1000500085BD86E083BD089585B5806185BD089521
:1000600085B58F7C85BD0895F7DF89E48A95F1F722
:10007000F7DF089581E080936000089582E0809327
:100080006000089580916000813031F4EDDF81E4FB
:1000900093E00197F1F7E8DF80916000823041F44E
:1000A000E3DF82E692E00197F1F700C00000DCDFB9
:1000B00010926000089581B3837F81BB82B38C600E
:1000C00082BB08954091610080B3242F30E090E01E
:1000D000809590958C7090702817390719F01092C0
:1000E00062000BC080916200813089F0813028F07D
:1000F000823011F1833081F52BC010926400109290
:100100006300442349F181E08093620025C080911F
:100110006300909164000196909364008093630063
:10012000442319F423E02093620084309105A0F069
:1001300082E08093620010C0483009F49BDF809118
:100140006100843009F49ADF83E08093620004C088
:10015000442311F41092620080B380958C708093D8
:100160006100811131D008951F920F920FB60F9246
:10017000112400000F900FBE0F901F9018951F9232
:100180000F920FB60F92112400000F900FBE0F9028
:100190001F9018950BD08FDF57DF94DF73DF19D0D6
:1001A00081E794E00197F1F70000F7CF87B3876309
:1001B00087BB84B38F6384BB81B3836F81BB85B7F7
:1001C000806285BF78940895109266001092650051
:1001D000089580916500909166009C012F5F3F4FCC
:1001E00030936600209365008233910570F0109281
:1001F0006600109265008BB7806C8BBF85B78068F6
:1002000085BF88958BB78F738BBF0895F894FFCF08
:00000001FF
